:10000000022291EFB40A07740D12000E740A3098A0
:1000100011A899B8130CC2983098FDA899C298B845
:1000200011F63099FDC299F599228E198F188C1C02
:100030008D1BE4F51DF51EF51FC0D043D01812DF4F
:10004000F94004D0D0D322D0D0C3228F18C0D043DF
:10005000D0180000000000000012DFF64004D0D0ED
:10006000D322D0D0C3223098FDAF99C2987E00220F
:10007000C287220238010203BEE86480F8E933E84F
:100080003360110460F0ED33EC337009E8FCE9FDF6
:10009000EAFEEBFF220460DED3EB9FEA9EE99DE8D7
:1000A000C2E78CF0C2F795F0400CE8CCF8E9CDF946
:1000B000EACEFAEBCFFB12038985D0F05804700327
:1000C00020D5B3E80470075002B2D50203C892D518
:1000D000EC0460F7E4CCC0E0C398F8603B9418608F
:1000E00008400DD0E0FB0203A0E4FBFAC9FC802825
:1000F000E830E406E4C9FBE4CAFCE830E305E4C9FF
:10010000CACBFCE854076010F8C3E913F9EA13FA04
:10011000EB13FBEC13FCD8F130F52FC3E49CFCEFA0
:100120009BFFEE9AFEED99FDD0E0FBEF4E4D4C703B
:100130001222DB030203C5EC2CFCEF33FFEE33FE8F
:10014000ED33FDED30E7EB0203A0EF2BFFEE3AFEBF
:10015000ED39FDD0E0FB50130BBB00030203C8EDEB
:1001600013FDEE13FEEF13FFEC13FC0203A0EC4DA6
:100170006011E8497017ED33EC3304600DE4FCFFC7
:10018000FEFD22E933E8330470F80203BE1203894E
:1001900058046009E4CC248150062850090203C8A1
:1001A0002840030203C5C0E0EB4A7044B98006D082
:1001B000E0FB0203B4EF4E701CBD8008EBFFEAFECB
:1001C000E9FD80EBE98DF0A4FEE5F0020257E9CDF0
:1001D000F9EAFEEBFFEF89F0A4FCE5F0CE89F0A48C
:1001E0002EFFE435F0CD89F0A42DFEE435F08067D4
:1001F000EF4E7005BD80D780C3EF8BF0A4ACF0EE5E
:100200008BF0A42CFCE435F0F8EF8AF0A42CE5F098
:1002100038FCE433CB8DF0A42CFCE5F03BF8EE8AFF
:10022000F0A42CFCE5F038F8E433CF89F0A42CFCE2
:10023000E5F038CF3400CE89F0A42FFFE5F03EFE84
:10024000E433C98DF0A42EFEE5F039CD8AF0A42F59
:10025000FFE5F03EFEE43DFD33D0E0FB50070BBB75
:10026000000F0203C8EC2CFCEF33FFEE33FEED333E
:10027000FD0203A00203C8EC5D046005E8590470A8
:10028000030203BE120389580460F6EC4860F2ECE6
:100290007004FDFEFF22C860DB2481C85009C398AA
:1002A000600250060203C59850CAF582E9294B4AFC
:1002B0007005AB820203B475F0007C1A7880C3EF3E
:1002C0009BEE9AED99400DC3EF9BFFEE9AFEED99E0
:1002D000FDE842F0DC23ACF0D0E0FFD0E0FED0E05F
:1002E000FDAB8220E7101BEB60BAEC2CFCEF33FF78
:1002F000EE33FEED33FD0203A0E803F830E705C05E
:10030000F075F000EF2FFFEE33FEED33FD40B83017
:10031000E7C280AA75F020800E75F010800575F098
:10032000087D007E007F003392D530D50312077F11
:10033000EC334010EF33FFEE33FEED33FDEC33FCD6
:10034000D5F0ED22E5F0247EA2D513CC92E7CDCEF8
:10035000FF22EDD2E7CD33EC3392D524814006E481
:10036000FFFEFDFC22FCE4CFCECDCC24E050117486
:10037000FF80EDC3CC13CCCD13CDCE13CECF13CF96
:100380000470F030D5DE02077FE9D2E7C933E833E5
:10039000F892D5EDD2E7CD33EC33FC5002B2D52242
:1003A000EC30E7100FBF000C0EBE00080DBD0004BE
:1003B0000BEB6014A2D5EB13FCED92E7FD2274FF6A
:1003C000FCFDFEFF22E480F8A2D574FF13FC7D80C3
:1003D000E480EFF920E73624F950037907E4F424A8
:1003E00002FBE582158270021583DBF6E024FB50E8
:1003F0001BE96014E4F0E582158270021583E004C5
:10040000F0B40A08E4F0D9EE7401F00A22C2D52251
:10041000ED33EC3392D5FA602AB4FF33EDC2E77BBB
:10042000FF60067A047935E4227A04793E20D50407
:100430007A047939224E614E002B494E46002D49EF
:100440004E4600E47A08F0A3DAFC7B00740722C071
:1004500083C082ECC0E0EDC0E0EEC0E0EFC0E0EAB7
:1004600075F010A4CAABF075F04DA42BFBE435F089
:10047000FCEA2410FAEB34C5FBEC34D9FCEDC2E7FE
:10048000FF75F056A4F42411C5F0F434C58FF0A420
:100490002AE5F03BE43CF020E714120556D0E0FFDB
:1004A000D0E0FED0E0FDD0E0FC1202778014F4042E
:1004B000120556D0E0FFD0E0FED0E0FDD0E0FC1207
:1004C000016ED082D083E0FAEDD2E7CD33EC332455
:1004D00082FBE4C3CF33CFCE33CECD33CD33DBF38A
:1004E0007B0775F00A846004F0A31B0AE5F0F0A313
:1004F0008FF0740AA4FFACF08EF0740AA42CFEAC4A
:10050000F050010C8DF0740AA42CFDE435F0F0A33A
:10051000DBDE740722ED33EC33600A047003BD8028
:1005200004ECB2E7FC223F8000004120000042C8FA
:100530000000447A0000461C400047C35000497444
:1005400024004B1896804CBEBC205A0E1BCA675321
:10055000C21C749DC5AEFB60065407601C232312A9
:100560000584EB5438600912057012057F12016E84
:10057000ECF8EDF9EEFAEFCB22EB12057F80F154A7
:100580003803241C900526FE93FC0EEE93FD0EEE20
:10059000930ECE93FF22BB010689828A83E022500C
:1005A00002E722BBFE02E32289828A83E49322BB14
:1005B000010CE58229F582E5833AF583E0225006B5
:1005C000E92582F8E622BBFE06E92582F8E222E56B
:1005D0008229F582E5833AF583E49322BB010689FB
:1005E000828A83F0225002F722BBFE01F322F8BB7D
:1005F000010DE58229F582E5833AF583E8F0225082
:1006000006E92582C8F622BBFE05E92582C8F2224A
:10061000EF8DF0A4A8F0CF8CF0A428CE8DF0A42EFE
:10062000FE22C5F0F8A3E028F0C5F0F8E5821582B7
:1006300070021583E038F022A3F8E0C5F025F0F051
:10064000E582158270021583E0C838F0E822BB010C
:100650000A89828A83E0F5F0A3E022500687F00938
:10066000E71922BBFE07E3F5F009E3192289828A24
:1006700083E493F5F074019322BB010789828A8396
:10068000020638500B09C5F027C7C5F01937C72235
:10069000BBFE0F09F8E3C5F025F0F319E3C838F302
:1006A000E82289828A83740193F5F0E49322BB01E6
:1006B00010E58229F582E5833AF583E0F5F0A3E0C1
:1006C000225009E92582F886F008E622BBFE0AE9F5
:1006D0002582F8E2F5F008E222E5832AF583E99322
:1006E000F5F0A3E99322BB010DC58229C582C5831C
:1006F0003AC5830206225011C58229F808E5F02682
:10070000F618F5F0E58236F622BBFE11C58229F80F
:1007100008E225F0F5F0F218E23582F222F8E582DF
:1007200029F582E5832AF58374019325F0F5F0E439
:10073000933822BB010A89828A83F0E5F0A3F02274
:100740005006F709A7F01922BBFE06F3E5F009F3FE
:100750001922F8BB0111E58229F582E5833AF58378
:10076000E8F0E5F0A3F0225009E92582C8F608A6D2
:10077000F022BBFE09E92582C8F2E5F008F222C3A7
:10078000E49FFFE49EFEE49DFDE49CFC22EB9FF5CC
:10079000F0EA9E42F0E99D42F0E89C45F022E860D4
:1007A0000FECC313FCED13FDEE13FEEF13FFD8F1B6
:1007B00022E8600FEFC333FFEE33FEED33FDEC3381
:1007C000FCD8F122BB010789828A830209335005D4
:1007D000E9F8020927BBFE05E9F802093F89828A88
:1007E0008302082EBB010DE58229F582E5833AF5E7
:1007F000830209335007E92582F8020927BBFE0767
:10080000E92582F802093FE58229F582E5833AF578
:100810008302082EBB010789828A8302084E500595
:10082000E9F802094BBBFE05E9F802095722E493F7
:10083000FC740193FD740293FE740393FF22E4930E
:10084000F8740193F9740293FA740393FB22ECF0A9
:10085000A3EDF0A3EEF0A3EFF022A8828583F0D001
:1008600083D082120871120871120871120871E4A3
:1008700073E493A3C583C5F0C583C8C582C8F0A33C
:10088000C583C5F0C583C8C582C822BB010DE582FA
:1008900029F582E5833AF58302085A5007E9258253
:1008A000F8020963BBFE07E92582F802097C22A44D
:1008B0002582F582E5F03583F58322E0FBA3E0FA9B
:1008C000A3E0F922F8E0FBA3A3E0F925F0F0E5822C
:1008D000158270021583E0FA38F022F8E0FBA3A33A
:1008E000E025F0F9F0E582158270021583E038FA10
:1008F000F022EBF0A3EAF0A3E9F022D083D082F853
:10090000E4937012740193700DA3A393F874019390
:10091000F5828883E4737402936860EFA3A3A380D5
:10092000DF8A838982E473E6FC08E6FD08E6FE08B8
:10093000E6FF22E0FCA3E0FDA3E0FEA3E0FF22E24D
:10094000FC08E2FD08E2FE08E2FF22ECF608EDF604
:1009500008EEF608EFF622ECF208EDF208EEF208E7
:10096000EFF222D083D082E493F608740193F60864
:10097000740293F608740393F6740473D083D082E0
:10098000E493F208740193F208740293F20874037A
:1009900093F27404730A0A2D2053657276696365B5
:1009A000204D6F6465202D20707265737320616E19
:1009B00079206B657920746F2073746172740A00FA
:1009C00065203D20657261736520636F72722066D9
:1009D00061630A0073203D2073696E676C65207344
:1009E00063616E0A0062203D20626F74746F6D2037
:1009F00031782070756C73650A0074203D20746F27
:100A0000702031782070756C73650A0069203D2074
:100A1000696E74657220626C6F636B203178207030
:100A2000756C73650A006D203D207363616E2B62E7
:100A3000616C616E63696E673220286D616E75202E
:100A40006D6F6465290A0075203D207363616E2B0C
:100A500062616C616E63696E673120286175746FC5
:100A6000206D6F6465290A0076203D207363616EF6
:100A70002B62616C616E63696E67322028617574E8
:100A80006F206D6F6465290A0079203D20736361D2
:100A90006E2B496E746572426C6F636B42616C6160
:100AA0006E63696E6720286175746F206D6F646571
:100AB000290A0063203D2063616C69627261746978
:100AC0006F6E2062792068616E640A0061203D20AB
:100AD00063616C6962726174696F6E20627920660D
:100AE000696C650A0020202020466F726D61743A9F
:100AF0002063686E5F302C2063686E5F312C202E7F
:100B00002E2E2E2C202063686E5F392C20426C6FB5
:100B1000636B2C20610A0064203D2074657374208F
:100B20006F6620536563732C205072696D4C206191
:100B30006E64205072696D48204D6F7366657473E2
:100B40000A006B203D206368616E676520434F4D4E
:100B500020737065656420746F2031392C32303019
:100B60006B0A006C203D206368616E676520434F0F
:100B70004D20737065656420746F203131352C32DF
:100B8000306B0A000A0A457261736520636F7272E6
:100B900020666163206D656D6F7279204030784208
:100BA0004645300A0A002D3E2031392C326B426115
:100BB00075640A002D3E203131352C326B4261754F
:100BC000640A000A20426F74746F6D42616C616E3A
:100BD00063696E672031782E2E2E20656E746572E3
:100BE000207468652063656C6C2063686E2E202815
:100BF000302D3131293A2000256275002070726550
:100C0000737320616E79206B657920746F20726533
:100C100070656174206F72204553430A000A457362
:100C2000636170652E2E2E2E2E0A000A20546F70DE
:100C300042616C616E63696E672031782E2E2E20C2
:100C4000656E746572207468652063656C6C2063E2
:100C5000686E2E2028302D3131293A20000A204993
:100C60006E746572426C6F636B42616C616E636936
:100C70006E672031782E2E2E20656E74657220747A
:100C800068652063656C6C2063686E2E2028302DAB
:100C90003131293A20000A2057726974652F526554
:100CA000616420666C6173686564206572726F723E
:100CB00073202F204553430A000A2053696E676C46
:100CC00065207363616E2E2E2E0A0020546F7020F3
:100CD0002F20426F74746F6D202F20496E746572DF
:100CE0002042616C616E63696E672028742F622FE9
:100CF00069293A20002563000A2042616C616E6315
:100D0000696E672031782E2E2E20656E74657220F4
:100D10007468652063656C6C2063686E2E202830D3
:100D20002D3131293A20000A205363616E2B426134
:100D30006C616E63696E672E2E2E2873656C656319
:100D400074206D6F6465290A006661756C740A0011
:100D50000A205363616E2B42616C616E63696E673A
:100D6000312E2E2E286E6F726D616C206D6F646552
:100D700029202F204553430A000A205363616E2B1C
:100D800042616C616E63696E67322E2E2E286E6F23
:100D9000726D616C206D6F646529202F204553436F
:100DA0000A000A496E746572426C6F636B42616C33
:100DB000616E63696E672E2E2E286E6F726D616C88
:100DC000206D6F646529202F204553430A0A006770
:100DD000657420203C2D2055626C6F636B3A25357D
:100DE0002E3366560A0A00496E746572426C6F6350
:100DF0006B3A256275205B313D7965732C20303D5F
:100E00006E6F5D0A0A0073656E64202D3E20000A35
:100E10002043616C6962726174696F6E206279202F
:100E200066696C650A000A0A726563656976652001
:100E30006368616E6E656C206461746120737472A6
:100E400065616D3A0A002566000A000A676F275B34
:100E50002562755D3A252E34660A00676F275B258B
:100E600062755D3A252E33660A00446F20796F75EE
:100E70002077616E7420746F20666C6173682079CE
:100E80002F6E3F0A006572726F72202D2063616CB5
:100E90002E6661632E2063686E2E256264202121F8
:100EA000210A006572726F72202D2063616C2E66BC
:100EB00061632E20626C6F636B3A202121210A004E
:100EC00043616C6962726174696F6E20636C6F73E9
:100ED00065640A002055626C6F636B6469673A252C
:100EE0003464200A002055626C6F636B3A25352EFE
:100EF0003366560A0A00456E746572207468652070
:100F0000626C6F636B20766F6C746167653A007614
:100F1000616C756520252E3366200A00676F275B9C
:100F20002562755D3A252E34660A000A2043616CFD
:100F30006962726174696F6E2062792068616E64A3
:100F40000A00456E74657220746865202562752EEE
:100F50002063656C6C2063686E2E3A000A2A2A2A88
:100F60005465737420616C6C20536563732A2A2A5C
:100F70000A002533643C3230202D3E205365632522
:100F8000626420696E6163746976650A0025336462
:100F90003E3230202D3E205365632562642061631C
:100FA000746976650A000A2A2A2A546573742050E7
:100FB00072696D4C2A2A2A0A002533643C3230209B
:100FC0002D3E20546573745072696D4C20666169C2
:100FD0006C0A0A002533643E3230202D3E205465D1
:100FE00073745072696D4C20706173730A0A002A21
:100FF0002A2A54657374205072696D482A2A2A0A75
:1010000000312E202533643E32300A00322E202556
:1010100033643E3230200A002D3E2028322E2D31FE
:101020003030293E312E29205072696D482061638D
:10103000746976650A0A002D3E2028322E2D313043
:1010400030293C312E29205072696D4820696E612B
:1010500063746976650A0A001B5B324A001B5B32C7
:101060003B3248000A002A2A2A2A2A2A2A2A2A2A1D
:101070002A2A2A2A2A2A2A2A2A2A2A2A2A2A2A2AD0
:101080002A2A2A2A2A2A2A2A2A2A2A2A2A2A2A2AC0
:101090002A0A002D42415454455259204D414E4197
:1010A00047454D454E542025732025732D0A004D8C
:1010B000617920323520323031300031343A3330EA
:1010C0003A3031002D754320535720666F7220252A
:1010D000732C2025732D200A004131323320204209
:1010E0004D53202831302063656C6C732900424FCA
:1010F00041524476342E30002D434F4D207370659D
:1011000065643A2031392C326B426175642D0A00D6
:101110002D43414E2073706565643A20323530208E
:101120006B426175642D0A001B5B346D001B5B31E3
:101130006D000A4D6561737572656D656E743A0A6E
:10114000001B5B306D0020546D696E3A2537644397
:1011500020546D61783A25346443200A0020556D8F
:10116000696E3A25372E32665620556D61783A25DC
:10117000342E3266560A002055626C6F636B3A2536
:10118000352E3266560A0A002055646966663A258D
:10119000362E3266560A002055617665723A25363B
:1011A0002E3266560A0020556D696E3A25372E3369
:1011B000665620556D61783A25342E3366560A0AF4
:1011C000002054656D70313A25366443200A20545E
:1011D000656D70323A25366443200A2054656D707F
:1011E000333A25366443200A002054626F617264EA
:1011F0003A25356443200A0A00205530636F727225
:101200003A25352E336656200A00205531636F7219
:10121000723A25352E336656200A00205532636F08
:1012200072723A25352E336656200A0020553363F4
:101230006F72723A25352E336656200A00205534D7
:10124000636F72723A25352E336656200A00205598
:1012500035636F72723A25352E336656200A0020A8
:101260005536636F72723A25352E336656200A0062
:10127000205537636F72723A25352E336656200A31
:1012800000205538636F72723A25352E336656202A
:101290000A00205539636F72723A25352E3366562F
:1012A000200A0020553130636F72723A25342E3394
:1012B0006656200A0020553131636F72723A253428
:1012C0002E336656200A0A002055626C6F636B3A13
:1012D00025352E3366560A0A002055646966663A3B
:1012E00025362E336656200A002055617665723AFF
:1012F00025362E336656200A000A20553064696769
:101300003A253464200A002055316469673A25344F
:1013100064200A002055326469673A253464200A43
:10132000002055336469673A253464200A0020554B
:10133000346469673A253464200A002055356469AD
:10134000673A253464200A002055366469673A25D7
:101350003464200A002055376469673A25346420D4
:101360000A002055386469673A253464200A002051
:1013700055396469673A253464200A0020553130B4
:101380006469673A2533640A00205531316469671E
:101390003A2533640A002055626C6F636B64696799
:1013A0003A253464200A005354415445202D204EE0
:1013B0006F726D616C20532562640A00535441546E
:1013C00045202D2043656C6C436F6E20696E7661FD
:1013D0006C69640A005354415445202D204E6F20FF
:1013E000436F6D2C20532562642067657473206EF3
:1013F0006F20726571756573740A005354415445CA
:10140000202D20426C6F636B436F6E20696E766196
:101410006C69640A000A5354415445202D205265DA
:1014200073657420532562640A0053256264206842
:1014300061736E2774206265656E207265717565D3
:10144000737465640A00532562642063616E2774B7
:101450002073746172740A0A005374617465207594
:101460006E6B6E6F776E2121210A00457261736584
:1014700020536563746F7273203020616E64203175
:101480000A002054656D70313A25362E31664320AE
:101490000A2054656D70323A25362E316643200A93
:1014A0002054656D70333A25362E316643200A008C
:1014B0002054626F6172643A25352E316643200AEA
:1014C0000A00205530636F72723A25352E32665607
:1014D000200A00205531636F72723A25352E32662C
:1014E00056200A00205532636F72723A25352E322B
:1014F0006656200A00205533636F72723A25352EE6
:10150000326656200A00205534636F72723A2535D0
:101510002E326656200A00205535636F72723A25C6
:10152000352E326656200A00205536636F72723AA5
:1015300025352E326656200A00205537636F7272A9
:101540003A25352E326656200A00205538636F72D0
:10155000723A25352E326656200A00205539636FBF
:1015600072723A25352E326656200A0020553130E7
:10157000636F72723A25342E326656200A00205567
:101580003131636F72723A25342E326656200A0A60
:10159000000A494E54455220426C6F636B204261F1
:1015A0006C616E63653A2562640A000A2D2D2D0A6E
:1015B000000A546F7042616C616E63653A25626423
:1015C0000A000A426F74746F6D42616C616E6365EC
:1015D0003A2562640A00E508242CF582E434F1F52A
:1015E00083E005082290F12930080390F12CE4757E
:1015F000F0011208C40205962001E97F2ED2018075
:1016000018EF540F2490D43440D4FF30050BEF244E
:10161000BFB41A0050032461FFE5096002150905F3
:101620000CE50C7002050B30080E90F129E475F002
:10163000011208C4EF0205DC0200037403D2088023
:1016400003E4C208F50890F1291208F2E4F509F55F
:101650000BF50CE50960077F2012161980F5750A55
:10166000FFC202C201C203C204C206C207C20912FB
:1016700015E5FF700D3008057F0012162AAF0CAE7D
:101680000B22B4255FC2D5C2051215E5FF24D0B4E4
:101690000A00501A75F00A780930D50508B6FF011E
:1016A00006C6A426F620D5047002D20480D924CF21
:1016B000B41A00EF5004C2E5D20502191CD2028010
:1016C000C6D20180C0D20380BCD2D580BAD20680F7
:1016D000B47F201216192003077401B5090040F1E8
:1016E0001215D6FF121619021653D209D207809589
:1016F0001215D6FB1215D6FA1215D6F94A4B7006FA
:10170000791A7A1A7BFF20032EE509602A7E008E63
:10171000827583001205AF60060EEE650A70F0C296
:10172000D5EBC0E0EAC0E0E9C0E0EE12197DD0E000
:10173000F9D0E0FAD0E0FB120596FF60AAEBC0E01A
:10174000EAC0E0E9C0E0121619D0E02401F9D0E0C7
:101750003400FAD0E0FBE50A0460DCD50AD98087C2
:10176000D20380A212195F60F7E50A700104120328
:10177000D3A90A600DE50A600914F50A121A07EFE9
:1017800060F3EA30E702F404C3995079EAF4250AD9
:101790000430E701E404F50A800D12195F60C1EA24
:1017A000050A250A1203D3EA90F158F030E701E464
:1017B000250A04D50A042006011412197DE4C0E0AC
:1017C000121A0790F158E0601320E70714F0121680
:1017D00001802204F0D0E014C0E07F00121601E581
:1017E0000A60071215F8150A800B3006031215F867
:1017F000D0E0021653D0E00480C412195F609EE569
:101800000A041203D390F158EAF0E50A20060260B8
:101810000104240412197D74FF04C0E0121A071297
:101820001601E50A20060260031215F8D0E0B50A99
:10183000E87F4512160B90F158E07F2B30E7047FCC
:101840002DF404C0E0121619D0E075F00A84C0F03F
:10185000121602D0E0121602021653791080027995
:1018600008C207C2098008D2D5790A8004790AC261
:10187000D5E50A047002F50AE4FAFDFEFF1215D65A
:10188000FC7B082002131215D6FD7B1030010A12D2
:1018900015D6FE1215D6FF7B20EC3382D592D5509B
:1018A00013C3E43001069FFFE49EFEE42002039D83
:1018B000FDE49CFCE4CBF8C202EC700CCFCECDCCA6
:1018C000E824F8F870F38017C3EF33FFEE33FEED32
:1018D00033FDEC33FCEB33FB994002FB0FD8E9EB13
:1018E000300205F8D0E0C448B202C0E00AEC4D4E28
:1018F0004F78207B0070C2EAB50A0040BCC0E012FD
:10190000197FD0F0D0E0200204C4C0E0C4B202C00D
:10191000F0121602D0F0D5F0EB0216531208FB16A7
:10192000F053185B5816C14C16BD42185F4F18672C
:101930004418674916D643186D55179A4617FA4545
:101940001764471A3A5016C52D16C92E16EC2B16D9
:10195000CD2316EA201A232A168548000016E4E54E
:101960000AB4FF03750A061215D6FC1215D6FD122D
:1019700015D6FE1215D6FF90F151020410790AA275
:10198000D5200414300609B910020404B908010472
:10199000A2D52007025001042003689203B5090074
:1019A0005034C0E07F203004197F30A203720772E8
:1019B00006500F1219D6C203C207C206C2097F30F1
:1019C000800F300603E9C0E0121619300603D0E09C
:1019D000F9D0E0B509CC3006177F30B9100C1216DB
:1019E000197F583005077F788003B908031216194C
:1019F0003003057F2D0216197F202009F87F2B2048
:101A000007F322920380CF7F00B40700500B2451CC
:101A1000F582E434F1F583E0FF22286E756C6C29C1
:101A200000D2021215D63002F8C202780930D50170
:101A300008F60216852D504349581215D62403B4D2
:101A400005004001E4901A359312160A743A1216F2
:101A50000AD20475090402185BE50830030104F892
:101A600023282418F582E434F1F5832290F115300F
:101A7000030390F118E475F0011208C402059660A2
:101A8000EAC50C7002150B14C50C200304FF0223D9
:101A9000A090F11574FFF5F00208DBFF02237CE54E
:101AA000096006D509037F002220030F122368EF87
:101AB0006008050CE50C7002050B2290F115120868
:101AC000BB120596FF60E890F115E475F00112086D
:101AD000C480DC121AA9EFC0E0121A9BD0E040F3D8
:101AE000809DD2038002C20390F1151208F2E4F542
:101AF0000AF508F50BF50C750900C202C200C20117
:101B0000C204121A6CFF7005AF0A7E0022B42530A1
:101B1000121A6CFF24D0B40A00500C75F00AC509E3
:101B2000A42509F50980E924CFB41A00EF5002C2B8
:101B3000E5021D7FD20180D8D20080D4D20480D0AB
:101B4000EF121A9B5008121AD3EF600E80A9EFC053
:101B5000E0121AA9D0E06F609EEF6074121A7F80C5
:101B6000A7121AA9EF6069E5097007050980031239
:101B70001AA9EF601420040E121A59E475F001122C
:101B800008C4EF1205DCD509E62004040508050A9F
:101B900080BA121A9FEFC0E0121A9BD0E0500412D4
:101BA0001A7FE4FF20040E121A59E475F00112089E
:101BB000C4EF1205DCEF70DA2004040508050A8082
:101BC0008BE50960020509121AD3121A9FEF70C63D
:101BD000300304E4121A7FE50A6003021B087EFF4B
:101BE0007FFF22E50960020509121AD3D206D20549
:101BF000121A9FEF30060260D7C0E0121A7FD0E0C1
:101C0000AC0DAD0EAE0FAF101221BE8C0D8D0E8E31
:101C10000F8F105007121AA9C20580D4200410207B
:101C20000502050A121A591208BB05081208140207
:101C30001AF7D0E0809A7900800A79108006790836
:101C40008002790AD205E50960020509E9C0E012BF
:101C50001AD3EF60DD121AA9BF2D04D2028003BF90
:101C60002B09121AD3EF60CA121A9FD0E0B40A02ED
:101C70008033B40802802EBF302770027408C2057A
:101C8000C0E0121A9FD0E0BF78028003BF5816054B
:101C900009D509028007D50904D205800B7410808C
:101CA000197002740ABF000AEFF8E4FCFDFEFF029F
:101CB0001D32C0E0EF121A7FD0E0F9E4FCFDFEFF18
:101CC000E9C0E0ECC0E0EDC0E0EEC0E0EFC0E01243
:101CD0001A9FEFF8D0E0FFD0E0FED0E0FDD0E0FCAE
:101CE000D0F0E8604DB461004007B47B005002C200
:101CF000E524D0503DFA24F6500724F95034240A44
:101D0000FAEAB5F000502BCFA9F0A42FFF92D5E945
:101D1000C5F0CEA4A2D53EFE92D5E9C5F0CDA4A2D1
:101D2000D53DFD92D5E9C5F0CCA4A2D53CFCC205B9
:101D3000808EE8C0E020042A200508050A3002034E
:101D400012077F121A591208BB050820000B200148
:101D50000DEE8FF012073380091208148004EF1281
:101D600005DCD0E0121A7F021AF7200410121A596B
:101D70001208BB0508E50B850CF012073380E8124A
:101D800008FB1BC1531C3A581B384C1B34421B1018
:101D9000481C3E4F1C42441B61431C36491C4255A3
:101DA0001BE3461BE3451BE3471B3C2A1D6A4E0011
:101DB000001B40726561642066726F6D20466C6125
:101DC00073684164723A307825780A002D3E206E9F
:101DD00065787420656D70747920466C6173684114
:101DE00064723A307825780A001B5B33316D004508
:101DF00072726F723A2077726F6E6720666C6173D1
:101E00006820736563746F722121210A0A001B5BCD
:101E1000306D007772697474656E20746F20466C43
:101E20006173684164723A30782578200A005265FF
:101E3000616420666C6173686564204572726F72BC
:101E400073202830782578293A0A002D2043656CC4
:101E50006C4F7665724C6576656C3A20203078253B
:101E600062780A002D2043656C6C556E6465726C57
:101E70006576656C3A2030782562780A002D20540A
:101E8000656D704F7665726C6576656C3A202030B2
:101E9000782562780A002D20536C61766547657459
:101EA000734E6F50696E673A202562750A002D20C7
:101EB000426C6F636B556E6465724C6576656C3A07
:101EC000202562750A002D2054656D7053686F726D
:101ED000744375743A202020202562750A002D2055
:101EE00054656D704F70656E3A20202020202020B0
:101EF000202562750A000A626F6172642070617247
:101F0000616D6574657220666C61736865642040FC
:101F1000616464726573732030782578200A0A0042
:101F20000A5265616420466C6173682043616C2EBF
:101F3000204661632E3A0A002063616C2E6661635D
:101F40002E2063686E2E2562753A20252E34660A8F
:101F5000002063616C2E6661632E20626C6F636B80
:101F60003A20252E34660A0043F22301F16244F23E
:101F7000260000000041F1590442F15A000041F1ED
:101F80005E0041F161006024F2ABFF0070FF491F69
:101F9000FF4922FF4925FF4928FF492BFF492EFF12
:101FA0004931FF4934FF4937FF493AFF493D60480D
:101FB000F2CFFF493EFF4941FF4944FF4947FF49EE
:101FC0004AFF494DFF4950FF4953FF4956FF4959C0
:101FD000FF495CFF495FFF4962FF4965FF4968FFB0
:101FE000496BFF496EFF4971FF4974FF4977FF490B
:101FF0007AFF497DFF4980FF49834CF317FF5175F4
:10200000FF4F0EFF5072FF530C6020F22B0485042B
:102010008D0495049D04A504AD04B504BD04C50458
:10202000CD04D504DD04E504ED04F504FD6020F2E3
:102030004B0484048C0494049C04A404AC04B404F1
:10204000BC04C404CC04D404DC04E404EC04F404B0
:10205000FC6020F26B0487048F0497049F04A7049C
:10206000AF04B704BF04C704CF04D704DF04E704F8
:10207000EF04F704FF6020F28B000100020004006F
:102080000800100020004000800100020004000849
:1020900000100020004000800041F3230000536C3A
:1020A0006176653A2053657276696365206D6F6469
:1020B000650A001B5B33316D004572726F723A2006
:1020C0005563656C6C5B2562645D204F7665724C70
:1020D0006576656C0A001B5B306D004572726F722D
:1020E0003A205563656C6C5B2562645D20556E64B7
:1020F00065724C6576656C0A001B5B33326D005768
:1021000061726E696E673A2054256264204F706573
:102110006E0A005761726E696E673A2054256264D8
:102120002053686F72744375740A004572726F723F
:102130003A2054256264204F7665724C6576656C52
:102140002028363543290A004572726F723A2055AD
:10215000626C6F636B556E6465724C6576656C0A74
:10216000004572726F723A205072696D4C20696E30
:102170006163746976650A004572726F7254797092
:10218000653A203078256278204572726F72494432
:102190003A2030782562780A00536C6176653A20DF
:1021A000496E6974206F7665720A00C207C208C260
:1021B00009C20AF9E4F511F512FCFDFEFFE910066B
:1021C000EA20090CB42D04D209D322B42B02D32265
:1021D00024D0504794095041240A300A15F885123A
:1021E000F0740AA42872E74051C5F0704D85F012D2
:1021F000D322D208C0E0E4FBFA7920784112016EC4
:10220000ECF8EDF9EEFAEFFBD0E0FCE412031E125D
:10221000007D3007B41511D322240A200A20B4FE11
:102220000720071AD207D32224EB600424E0700EA3
:10223000A2099207D20AC209D322C30203BEE43024
:102240000A0BE512300902F404A20792093008EAE9
:10225000251120D2E5A2E7920A5002F404B4260028
:1022600050D8CCC0E0EDC0E0EEC0E0EFC0E0EC1232
:102270000556D0E0FFD0E0FED0E0FDD0E0FC200A23
:102280000512016E8003120277300903120515C38F
:102290002275BF0143B70843B70443B60453B6F7EA
:1022A000780AD9FED8FC43B602E5B620E1FB30E05F
:1022B000F543B70853B7FB75BB9853B70F43B7A0A7
:1022C00043B702E5B730E0FB53B7F775BF00787F3F
:1022D000E4F6D8FD90F0007F007E06E4F0A3DFFC7A
:1022E000DEFA75815D022323023FF5E493A3F8E44F
:1022F00093A34003F68001F208DFF48029E493A35E
:10230000F85407240CC8C333C4540F4420C8834076
:1023100004F456800146F6DFE4800B010204081045
:10232000204080901F68E47E019360BCA3FF543F6F
:1023300030E509541FFEE493A360010ECF54C0257D
:10234000E060A840B8E493A3FAE493A3F8E493A36D
:10235000C8C582C8CAC583CAF0A3C8C582C8CAC5D1
:1023600083CADFE9DEE780BE100B0B120066BF0DEB
:10237000027F0A02000390F324E0FF22EFC39409D6
:102380004005EF940E4004EFB42003D38001C32234
:10239000C0D0EF12DFF05004D0D0D322D0D0C3226F
:1023A00090F324EFF0D20B2275B201758644E4F568
:1023B000B27586B875B201759103F5B275917C75E9
:1023C000B1F375C90B2275BF0175BA10E4F5BF7181
:1023D000A81237F271ECF1F4910A122AD075B820E4
:1023E000E4F5B975F82075F930D2AF2275B2025311
:1023F00090FD439102E4F5B243910253B3FEF5BD63
:1024000075985075BE4D43BD012275A301E4F5A634
:10241000F5A7759C17F59D759E01F59F75A401F5AF
:10242000A5F5A3F59AF59BF59EF59F75A30275FAA0
:1024300001F5FBF5FEF5FFF5FCF5FDF5A7F59AF5C1
:102440009BF5A6F59EF59FF59CF59D75A303F5FFFD
:10245000F59EF59FF5A4F5A3759C40759D402290CF
:10246000F1307407F0E4FBFD7F01917F7F017E0076
:1024700075A3018E9D8F9CE480DCF0E4FBFDFFE4FE
:10248000FEEFB401027E80EDB4010474402EFEEB39
:10249000B4010474202EFE90F130E054072E75D163
:1024A00096F5D275D1D02290F11DF1EBE4A3F0A303
:1024B000F090F12AF0A3F090F130F0FBFDFF917F56
:1024C00090F1307401917A90F1307402917A90F128
:1024D000307403917AB1D2BFF1FB122864122893B1
:1024E00012289E90F126EEF0A3EFF01228BB90F197
:1024F00028EEF0A3EFF07FF1B1DB90F124B1E4D14D
:1025000039900042B1C290F126B1E4D13990004433
:10251000B1C290F128B1E4D139900046B1C290F136
:10252000307404917AB1D2BF11FB1228647F11B1CB
:10253000DB90F1307405917AB1D2BF21FB12289360
:102540007F21B1DBE490F12CF090F1307406917AA8
:10255000B1D2BF41FB12289E90F120EEF0A3EFF024
:1025600090F12BE02FF090F12AE03EF07F41B1DBBB
:10257000124203E0C36480948440CE12A4A5780282
:10258000CEC313CE13D8F9FF90F11DD1399000308E
:10259000B1C290F122B1E4D139900048B1C290F1BA
:1025A00024E0FFA3E090001ACF8FF01207529000B2
:1025B00030B1CB1249C390F11DD139900016B1C290
:1025C0000022EE8FF002075290001A1206AEFFAE04
:1025D000F02275D195AFCE75D1D02275D1958FCF20
:1025E00075D1D022E0FEA3E0FFB1EF90F11D2212E1
:1025F00049E375B7D175B66675B110E5B020E2FB59
:102600001249BBEF7806CEC313CE13D8F92414FFBA
:10261000EE34FFFE22439180D29790F00AE0FBA3B4
:10262000E0FAA3E0F912373690F00AE0FBA3E0FAF3
:10263000A3E0F912376690F00AE0FBA3E0FAA3E00A
:10264000F922F1E812A3EFF167D13990004C12366C
:102650006412A44D12366B7BFF7A117946F167D173
:102660003990003412379A1237E912084E90F1155A
:10267000D13990003212379A78451202771237AA70
:102680007BFF7A1179A6F167D13990004212366446
:1026900090004412A45012366B12A4BD90F1301277
:1026A000366B7BFF7A1179C1F167D13990004812FE
:1026B00036647BFF7A1179E9F167D13912064EF160
:1026C000747A1179F9F167D139900002F1717A12B7
:1026D000790AF167D139900004F1717A12791BF10E
:1026E00067D139900006F1717A12792CF167D139EE
:1026F000900008F1717A12793DF167D13990000AA2
:10270000F1717A12794EF167D13990000CF1717A3A
:1027100012795FF167D13990000EF1717A127970F8
:10272000F167D139900010F1717A127981F167D196
:1027300039F16E7A12799212164190F115D139124F
:1027400037977843F1827A1279C8F167D1399000CE
:1027500036F1717A1279D9F167D139900038F17177
:102760007A1279E902164112164190F11522900071
:10277000121206AEFDACF0E4120319E4FBFA798004
:10278000784512027790F12C12084E7BFF2290F0D0
:1027900007F1EBA3D1399000AE1205AFFF544C60A6
:1027A0000990F007D13974038033EF540360099026
:1027B000F007D13974018025D1369000AE1205AFF3
:1027C000FF30E40990F007D13974028010EF90F0E7
:1027D0000730E706D13974058003D139E41248CCBB
:1027E000D139E4F5F002073390F115EBF0A3EAF0EC
:1027F000A3E9F022E4F5D175CA1075CC5175D10169
:10280000F5CA75CB0175CC0275CD03F5CE75CF0138
:1028100075D20275D303F5D175CE0A75D10475CA88
:10282000C075CBC075CCC075CDC075D105F5CDF5E3
:10283000D3F5D175CDB775CF0275D10675CD05F538
:10284000CCF5D143CA8022116FE5CA30E412E5CA43
:10285000AECB7806CEC313CE13D8F9FFEE5403FEE9
:1028600075D1D022114790F122EEF0A3EFF022E4CF
:10287000FFFE75D19222116FE5CC30E412E5CCAEAB
:10288000CD7806CEC313CE13D8F9FFEE5403FE75F0
:10289000D1D022117690F124EEF0A3EFF022116F47
:1028A000E5CE30E412E5CEAECF7806CEC313CE131C
:1028B000D8F9FFEE5403FE75D1D022116FE5D23066
:1028C000E412E5D2AED37806CEC313CE13D8F9FF07
:1028D000EE5403FE75D1D022439C02F1FA1225D2A8
:1028E000BF81FA7F811225DB80D1E490F116F0A33D
:1028F000F0EF14607814700221912402600221DD4F
:102900007BFF7A0F795C121641E490F115F01224E6
:102910005FD2B7518690F2CF12A41A12263B120949
:1029200021439C02518690F2F312A41A12263B1204
:102930000921F1FA11DD5175F0C2B731F850137A5F
:102940000F797231E3517D12164190F116E004F0D7
:10295000800B7A0F798D31E3517D12164190F1157C
:10296000E004F0E0C36480948C40A380707BFF7A25
:102970000F79A612164112300B90F11831F3500660
:102980007A0F79B980047A0F79D431E31216418035
:102990004C7BFF7A0F79EF12164112245FD2B751A8
:1029A000015175F0C2B731F87A10790131E312168E
:1029B0004112245F510190F11A31F37A10790C9091
:1029C000F11A31E612164190F118E0FEA3E0FFA3E0
:1029D000E0FCA3E0FD12A00090F117EFF090F117DA
:1029E000E0FF2290F118E0FFA3E090F12CCFF0A3DC
:1029F000EFF022EEF0A3EFF0C39414EE94007BFF0F
:102A000022D2B6000000000000000000000000001C
:102A100000000000000000000000000000000000B6
:102A200000000000000000000000000000000000A6
:102A30000000000000000000000000000000000096
:102A40000000000000000000000000000000000086
:102A50000000000000000000000000000000000076
:102A600000000000000000C2B600000000000000EE
:102A700000000001D890F118EEF0A3EF2290F115BC
:102A8000E090F12EF02290F115E0FF3395E0FE2268
:102A900090F00AEFF0F1F3F1167D07F13051BC90A0
:102AA000F00A5189FDFCEF241012A489FC78101261
:102AB00007B1EF4402FFEC4402FC80047D087C0275
:102AC000D1CD75DC01E5DC30E00553D8FE80F6227F
:102AD000F1F375DC01E5DC30E00553D8FE80F675D6
:102AE000DA0075D98075DB4175D815E5D820E1FB92
:102AF00075DA0075D9C075DB4175D815E5D820E1C8
:102B0000FB75D804E4F5DB75DC6075D835E5D820B5
:102B1000E1FB75DB01E4F5DC75D835E5D820E1FB98
:102B200075DB4175DCD475D835E5D820E1FB75DD62
:102B30006075D845E5D820E1FBE4F5DBF5DCF5DD93
:102B400075D871E5D820E1FB75B20243B00843B1F6
:102B500008E4F5B243B108F5DA75D9717F02FEFDDC
:102B6000F1307D01F1307D02F1307D037C0251C0F6
:102B7000F1167D10F1307D11F1307D12F1307D13B1
:102B8000F1307D14F1307D15F1307D16F1307D1777
:102B9000F1307D18F1307D19F1307D1AF1307D1B57
:102BA000F1307D1CF1307D1DF1307D1EF1307D1F37
:102BB000F1307D07F13051BC75DA0475D907F14E5B
:102BC000F1107F007E007D207CD9D1F6F1397C3F69
:102BD000F1107F04D1FDF14075D90FF14EF1107F56
:102BE000007E007D247CD9D1F6F1397C3FF1107F45
:102BF000047E01D1FFF14075D917F14EF1107F002D
:102C00007E007D287CD9D1F6F1397C3FF1107F041C
:102C10007E02D1FFF14075D91FF14EF1107F007E89
:102C2000007D2C7CD9D1F6F1397C3FF1107F047EF8
:102C300003D1FFF14075D9277F007E007DA0F10E02
:102C400012A42B7CCCD1F6F1397C3FF1107F047EAD
:102C500004D1FF12A42B7C02F14875D92FF14EF15B
:102C60001012A42B7CC8D1F6F1397C3FF1107F04FF
:102C70007E05D1FF12A42B7C04F14875D937F14EA3
:102C8000F11012A42B7CD0D1F6F1397C3FF1107FEA
:102C9000047E06D1FF12A42B7C01F14875D93FF1C7
:102CA0004EF11012A493D1F6F1397C3FF1107F0060
:102CB0007E07D1FF12A42B7C02F14875D9477F0013
:102CC0007E007DA0F10E12A493D1F6F1397C3FF184
:102CD000107F007E08D1FF12A42B7C02F14875D929
:102CE00087F14EF1107F007E007D20D1F4F1397C18
:102CF0003FF1107F007E10D1FFF14075D98FF14E6A
:102D0000F1107F007E007D24D1F4F1397C3FF11079
:102D10007F007E11D1FFF14075D997F14EF1107F00
:102D2000007E007D28D1F4F1397C3FF1107F007ED8
:102D300012D1FFF14075D99FF14EF1107F007E0056
:102D40007D2CD1F4F1397C3FF1107F007E13D1FF4F
:102D5000F14075D9A7F14EF1107F007E007D30D192
:102D6000F4F1397C3FF1107F007E14D1FFF1407502
:102D7000D9AFF14EF1107F007E007D34D1F4F139EE
:102D80007C3FF1107F007E15D1FFF14075D9B7F17E
:102D90004EF1107F007E007D38D1F4F1397C3FF197
:102DA000107F007E16D1FFF14075D9BFF14EF110B2
:102DB0007F007E007D3CD1F4F1397C3FF1107F0033
:102DC0007E17D1FFF14075D9C7F14EF1107F007E1B
:102DD000007D40D1F4F1397C3FF1107F007E18D1A5
:102DE000FFF14075D9CFF14EF1107F007E007D4498
:102DF000D1F4F1397C3FF1107F007E19D1FFF14011
:102E000075D9D7F14EF1107F007E007D48D1F4F1E5
:102E1000397C3FF1107F007E1AD1FFF14075D9DF78
:102E2000F14EF1107F007E007D4CD1F4F1397C3FF2
:102E3000F1107F007E1BD1FFF14075D9E7F14EF113
:102E4000107F007E007D50D1F4F1397C3FF1107F7E
:102E5000007E1CD1FFF14075D9EFF14EF1107F00DB
:102E60007E007D54D1F4F1397C3FF1107F007E1D4E
:102E7000D1FFF14075D9F7F14EF1107F007E007D52
:102E800058D1F4F1397C3FF1107F007E1ED1FFF163
:102E90004075D9FFF14EF1107F007E007D5CD1F4CA
:102EA000F1397C3FF1107F007E1FD1FF12A42B7CF3
:102EB00008D1CD75DA0075D9C0E4F5D8E5D820E1A0
:102EC000FB53DBBE75D811E5D820E1FB2290F00B57
:102ED00012084E90F00EE0F5DB90F00DE0F5DC907E
:102EE000F00CE0F5DD90F00BE0F5DE75D8F1E5D8FB
:102EF00020E1FB227CDDD1CD75D8087F007E007DEE
:102F0000007C00D1CD75D8087F007E007D007C005C
:102F1000D1CD75D808227F027E007D047C0251C08D
:102F20007F027E007D057C0251C07F027E007D060F
:102F30007C0251C07F027E00227FFF7EFF7DFF2248
:102F40007F007E007D007C08D1CD75DA04227F00F1
:102F50007E007DA87C0E22F1F37F027E007D007C46
:102F600000F1327D017C00F1327D027C00F1327D86
:102F7000037C00F1327D047C00F1327D057C00F1A0
:102F8000327D067C00F1327D077C00F1327D087CC9
:102F900000F1327D107C00F1327D117C00F1327D38
:102FA000127C00F1327D137C00F1327D147C00F143
:102FB000327D157C00F1327D167C00F1327D177C6C
:102FC00000F1327D187C00F1327D197C00F1327DF8
:102FD0001A7C00F1327D1B7C00F1327D1C7C00F1FB
:102FE000327D1D7C00F1327D1E7C00F1327D1F7C24
:102FF0000041C075DA0075D9712275A391E5A6204C
:10300000E4FB75A3D0E5CB20E1FB2212245FD2B70D
:10301000D28300000000000000000000000000005B
:1030200000C283C2B70228D8110BC3EF9414EE94E8
:10303000005002C322D32290F1261227EB11284020
:103040002490F126319224AE118E44081205DC90B2
:10305000F1261185B1B67BFF7A217961B13B79D632
:10306000121641C32290F126319224AE118E54F7EC
:103070001205DC90F126118554FE1205DCD32212D4
:1030800005DC90F118E0FBA3E0FAA3E024B0F9E43A
:103090003AFA02059690F1181227EB90F1181226D1
:1030A0003990004A1206AED39418E5F064809481FA
:1030B000401EE924AF118E4402F1B7122639900068
:1030C00056B1317A2079FFB13B79D6121641800E84
:1030D00090F118319224AF118E54FD1205DC90F15D
:1030E0001812263990004C1206AEC39424E5F06401
:1030F00080947F501EE924AF118E4401F1B712264F
:1031000039900059B1317A217913B13B79D6121631
:1031100041800E90F118319224AF118E54FE1205A9
:10312000DC90F11812263990004A1225CBD3944135
:10313000EE64809480402BEF940EEE648094815076
:1031400021E924AE118E4404117FB1B690F118121A
:103150002639900056B1317A21792BB13B79D612BC
:10316000164190F118122639F1C7D39400E5F09476
:10317000195018E924AE118E4440117FB1B67BFF7F
:103180007A217948B13B79D6121641221216419024
:10319000F00AE0FBA3E0FAA3E02290F0071227EB8D
:1031A000E4A3F0FDFC90F007122639123B595002BF
:1031B000414275DA0475D927E4F5D8E5D820E1FB5A
:1031C000F1E130E06990F007319224AE118E54EFB6
:1031D000F1B0118554FB1205DC75DA0475D924E4CD
:1031E000F5D8E5D820E1FBACDCADDB90F00712268A
:1031F0003990005A1205AF123CD5748B2FF58274AA
:10320000F23EF583E05CFEA3E05D4E90005B60045F
:1032100074018001E41205EE75DA0475D92775DBB7
:103220000175D811E5D820E1FBAE04AF052290F07E
:1032300007319224AE118E4410F1B011854404126E
:1032400005DCE4FEFF2290F0021227EBE4A3F0A3DA
:10325000F0439180D29790F159E0146058147002B5
:1032600041E91470026113147002613C1470026130
:10327000692405600261AB90F002122639B12E7A02
:103280001379A7B127122639F13690F002122639A8
:10329000F16690F002122639F153122639319A90D4
:1032A000F002122639123B6590F002122639C20054
:1032B0001243506198D292C2967BFF7A1379BCB1C7
:1032C00027122639F16690F002122639F1531226A0
:1032D00039C20012435090F002F15E90F00AC91218
:1032E00027ECB1C412482D61B4C292D29690F0027C
:1032F000122639B12E7A1379D5B127122639319A8F
:1033000090F002F15E90F00AC91227ECB1C41248A5
:103310008061B4C292C2967BFF7A1379FBB1271207
:103320002639F13690F002122639F153F15E90F011
:103330000AC91227ECB1C41248D3807890F0021267
:103340002639B12E7A147915B127122639F1369023
:10335000F00212263912392A90F002122639123858
:10336000E390F002122639F13690F002122639125B
:103370003F1BEF702390F00212263912386A90F04A
:1033800002122639B12E7A14792AB127122639B1C0
:103390002E7A14794612164190F002F15E90F00AEE
:1033A000C91227ECB1C412278E80097BFF7A1479E9
:1033B0005912164190F0021226399000AEE412051F
:1033C000EE9000B0E41205EE53BCFD209802A12659
:1033D000C298E59964657025F1D97F041223905055
:1033E000F9125FDD7F0412239050F990F00212264B
:1033F0003912A1F57BFF7A14796B121641E59964B5
:10340000706002A10F90F002122639900042B1AF15
:10341000EC12031990F12C12084E90F0021226398A
:10342000900044B1AFEC120319F1AA90F0021226F9
:1034300039900046B1AFEC12031990F13412084EE6
:103440007BFF7A147982B127122639900048B1AFF8
:10345000EC1203191227857A1479B0B12712263994
:1034600012064E1227747A1479C2B12712263990A7
:1034700000021227717A1479D3B1271226399000ED
:10348000041227717A1479E4B127122639900006C4
:103490001227717A1479F5B1271226399000081293
:1034A00027717A157906B12712263990000A12275A
:1034B000717A157917B12712263990000C122771ED
:1034C0007A157928B12712263990000E1227717AC1
:1034D000157939B1271226399000101227717A1503
:1034E000794AB12712263912276E7A15795BB127EE
:1034F0001226399000141227717A15796CB12712AF
:1035000026399000161227717A15797E121641E538
:1035100099B4721290F00212263912A1F590F002BD
:1035200012263912425D2212164190F002229000BA
:103530005A1205AF90F12CF07BFF221216417BFF4F
:103540007A202290F1181227EB90F118122639F107
:10355000CDD39499E5F094394021E924AE118E44FD
:1035600001117FB1B690F1181226399000A4B13143
:103570007A2079B9B13B79D612164190F11812260A
:1035800039F1D3C3E5F094285021E924AE118E44DB
:1035900002117FB1B690F1181226399000ADB13109
:1035A0007A2079DBB13B79D6121641229000701255
:1035B00006AEFDACF02244011205DC7BFF7A2079D7
:1035C000B3021641A37401F0A374F1F0A3745AF08E
:1035D0007B017AF179592290F0071227EB12A3EFC1
:1035E00012164190F00712263990004CD16412A4B3
:1035F0004DD16B7BFF7A11794612164190F007127C
:103600002639900034F19AF1E912084E90F0071231
:103610002639900032F19A7845120277F1AA7BFFA1
:103620007A11795D12164190F007122639F19778D8
:10363000431227827A11797712164190F0071226E9
:10364000399000361227717A11798812164190F05C
:10365000071226399000381227717A1179970216CD
:10366000419000BB1206AEFF90F12CE5F0F0A3EF05
:10367000F0221227E890F11512263990001CD1642F
:103680007BFF7A1279F912276712263990001ED132
:10369000647BFF7A1379071227671226399000207E
:1036A000D1647BFF7A1379141227671226399000B0
:1036B00022D1647BFF7A1379211227671226399071
:1036C0000024D1647BFF7A13792E122767122639E2
:1036D000900026D1647BFF7A13793B12276712266C
:1036E00039900028D1647BFF7A137948122767123A
:1036F000263990002AD1647BFF7A13795512276707
:1037000012263990002CD1647BFF7A13796212273C
:103710006712263990002ED1647BFF7A13796F12DD
:10372000164190F115122639900030D1647BFF7A52
:103730001379960216411227E890F11512263912D4
:103740005F0690F115122639123C1F90F1151226D2
:10375000390195B1D790F00222F583E0F8A3E0F9A2
:10376000A3E0FAA3E0221227E890F11512263911FE
:1037700037502390F1151226391249F290F11512A3
:10378000263912A09D90F115122639124E0190F1A2
:1037900015122639B143229000161206AEFDACF088
:1037A000E4120319E4FBFA79802290F13002084E0A
:1037B0001205DC90F007221205DC7BFF7A2079F9F4
:1037C00012164190F118229000160206AE900032B7
:1037D0000206AE9000340206AE7D02FCFFFE02003F
:1037E0002A90F00AE5DBF0E022784512027790F1AA
:1037F0002C2275BB72E4F5A8F5E8F5B7F5BAF5B378
:1038000022C0E075BF00E5BC30E10353BCFDE5BC60
:1038100030E40353BCEFE5BC30E50353BCDFE5BC4B
:1038200030E60353BCBFD0E032E5D820E1FBC0D97D
:10383000C0DAC0DBC0DCC0DDC0DEEF75F008A42458
:1038400007FFE5F03404F5DA8FD9E4F5DCF5DB7534
:10385000DE0775DD2075D8F1E5D820E1FBD0DED09C
:10386000DDD0DCD0DBD0DAD0D92290F0101227EBFB
:1038700090F010122639715940629000AE1205AFD7
:10388000700411DD60561235BB90F010122639110C
:10389000DD90F12CF09000AE1205AF90F12DF07B91
:1038A000FF7A21797812353B79D612164175DA0400
:1038B00075D92C90F0101226399000AE1205AFF594
:1038C000DB11DDF5DC90005A1205AFF5DDE4F5DE25
:1038D00075D8F1E5D820E1FB7F051129229000B0D1
:1038E0000205AF90F0071227EBA37401F090F007E8
:1038F0001226397159402A7BFF7A21799912164193
:1039000075DA0475D93490F007122639312290F017
:103910000AE02FF5DB75D811E5D820E1FB7F061111
:10392000292290005A1205AFFF2290F0071227EBD0
:1039300090F00712263990001A1206AEC394DFE504
:10394000F09403402290005A74FF1205EE7BFF7A38
:1039500020799E121641122F577FF0122A9090F074
:103960000712263912532690F0071226391225C85D
:10397000C374A09F74039E500FC3EF94DFEE9403B3
:10398000500690005AE4614090F007122639122543
:10399000C8C374669F74039E500FEF94A0EE940307
:1039A000500790005A7401614090F00712263912B6
:1039B00025C8C374379F74039E500FEF9466EE942E
:1039C00003500790005A7402614090F007122639A4
:1039D0001225C8C3740C9F74039E500FEF9437EEEA
:1039E0009403500790005A7403614090F007122628
:1039F000391225C8C374E39F74029E500FEF940CD4
:103A0000EE9403500790005A7404614090F007123E
:103A100026391225C8C374BE9F74029E500FEF94BE
:103A2000E3EE9402500790005A7405614090F0074D
:103A30001226391225C8C374A09F74029E500FEF3E
:103A400094BEEE9402500790005A7406614090F0C4
:103A5000071226391225C8C374839F74029E500F23
:103A6000EF94A0EE9402500790005A7407614090C2
:103A7000F0071226391225C8C374669F74029E503F
:103A80000FEF9483EE9402500790005A740861403F
:103A900090F0071226391225C8C3744E9F74029EF7
:103AA000500FEF9466EE9402500790005A7409612B
:103AB0004090F0071226391225C8C374379F74024C
:103AC0009E500FEF944EEE9402500790005A740AE5
:103AD000806E90F0071226391225C8C374239F7494
:103AE000029E500FEF9437EE9402500790005A74E4
:103AF0000B804D90F0071226391225C8C3740E9F13
:103B000074029E500FEF9423EE9402500790005AD7
:103B1000740C802C90F0071226391225C8C374FC4F
:103B20009F74019E500FEF940EEE94025007900088
:103B30005A740D800B90F00712263990005A740EBB
:103B40001205EE122F5790F0071226393122122A51
:103B50009090F007122639212290005A1205AFC327
:103B6000648094802271595002810D1237D3AEF0D7
:103B70007807CEC313CE13D8F99000B11205EE1218
:103B800037CDAEF07807CEC313CE13D8F99000B27C
:103B90001205EE90004C1206AEFF9000B391189003
:103BA000004A1206AEFF9000B591181237C7FF9079
:103BB00000B7911890005A1205AF91D5744B2FF5AC
:103BC0008274F2F1138EDAF5D99000B21205AFF5D6
:103BD000DB9000B11205AFF5DC9000B3D1F3E5D86E
:103BE00020E1FB90005A1205AF91D5742B2FF5827E
:103BF00074F2F1138EDAF5D99000B51206AE85F0A5
:103C0000DCF5DB9000B7D1F3E5D820E1FB22900092
:103C1000B91206AEFF9000BBE5F08FF0020752909C
:103C2000F1181227EB90F118122639900042120673
:103C3000AEFF90004E911890005674011205EE9060
:103C400000441206AEFF9000509118900057740285
:103C50001205EE12A4BD9000529118900058740302
:103C60001205EE9000481206AEFF90005491189095
:103C7000005974041205EEE9244EF9E43AFAC0033F
:103C8000C002C00190F1181231922456124F061250
:103C900027EBA37404F0D001D002D003B14990F116
:103CA0001812263990004E1206AEFF90004A911865
:103CB0009000541206AEFF90004CE5F08FF0020722
:103CC0005290F118E0FBA3E0FAA3E0241CF9E43AD7
:103CD000FA90F22AE0FF3395E0FEEF25E0FFEE33A5
:103CE000FE2290F126EFF0AF05E4FCA304F0A374EC
:103CF000F2F0A37426F0EF24BE602624EE7042E4B6
:103D0000FDED91D590F127122639D1FFB5070BEDC6
:103D100091D5D115D1DAB442010C0DEDB402E28097
:103D200020E4FDED91D590F127122639D1FFB5079A
:103D30000BED91D5D115D1DAB454010C0DEDB402CF
:103D4000E2EC7F0060027F012290F11B1227EB90D2
:103D5000F1227401F0E4A3F090F121E014FF90F15E
:103D600023D1E74002C10FE4A3F090F122E0FF90DD
:103D7000F121E0C39FFF90F124D1E74002C108EE9A
:103D800091D590F11B123192F1CB1235AF90F11B0E
:103D900012263BD1E0FFD3ED9FE5F06480F8EC64A0
:103DA0008098405C90F12491D4D1E0FD90F126F10F
:103DB0000CD1159000021206AEFD90F12491D49022
:103DC000F11B12263BF1C212075290F126D110F1DD
:103DD000B990F11E12263990F124122A898F82F5AA
:103DE000831205AF90F125F0D115D1DAFF90F11EC5
:103DF00012263B90F124F1E190F125F1D41205EE69
:103E000090F124E004F0A16A90F122F1B1A15822CE
:103E1000E0FCA3E0FDE92FF9EA3EFA2290F124123A
:103E200027EB90F12B7401F0E4A3F090F12AE01459
:103E3000FF90F12CD1E74002C1D9E4A3F090F12B1F
:103E4000E0FF90F12AE0C39FFF90F12DD1E74002FF
:103E5000C1D2EE91D590F124123192F1CB1235AF4F
:103E600090F12412263BD1E0FFD3ED9FEC95F0407A
:103E70005C90F12D91D4D1E0FD90F12FF10CD11592
:103E80009000021206AEFD90F12D91D490F1241213
:103E9000263BF1C212075290F12FD110F1B990F1E7
:103EA0002712263990F12D122A898F82F583120567
:103EB000AF90F12EF0D115D1DAFF90F12712263B09
:103EC00090F12DF1E190F12EF1D41205EE12424F56
:103ED000C13D90F12BF1B1C12B229000010205AF41
:103EE0008F828E830206AEE0FEC3EF6480F8EE643C
:103EF0008098221206AE85F0DEF5DD75D8F1228FAE
:103F0000828E831205AFFF90F126E022E5F0F0A348
:103F1000EDF0223EF583E0FEA3E02290F0071227A9
:103F2000EBE4A3F090F007122639715950037F019A
:103F30002290F00B12085A00000000E47F507EC36C
:103F4000FDFC90F00B12375BFBC312078D504790BE
:103F5000F00712263990005A1205AF91D5746B2FD5
:103F6000F58274F2F1138EDAF5D9E4F5D8E5D820AC
:103F7000E1FB1237E130E0037F012290F00BE0FC1F
:103F8000A3E0FDA3E0FEA3E0240112A489FC90F0CD
:103F90000B12084E80A590F00712319224AE123019
:103FA0008E44801237B012308544041205DC7F0045
:103FB00022E004F0A3E004F022900002EC8DF00275
:103FC00007528F828E83E5F08DF0222FF9EA3EFAB8
:103FD00090000222E0FFE92DF9EA3CFA900001EF9F
:103FE00022E0FD3395E0FC8D82F583EF0205EE11B2
:103FF0006A90F00D221223C6D29912417C7A107970
:104000005D121641E490F1BDF090F000F0A3F09045
:10401000F000E0FEA3E0FFC3940AEE9400501C9071
:10402000F2AB12A41A12263B12092190F001E0040F
:10403000F0700690F000E004F080D4C2B753BCFDED
:104040007BFF7A107964121641317C7A10796431E1
:104050007090F12C74FFF0A37410F0A374AF316969
:104060007410F0A374BBF07BFF7A107993121641A1
:1040700090F12C74FFF0A37410F0A374D93169741B
:1040800010F0A374EEF07BFF7A1079C41216417B16
:10409000FF7A1079F81216417BFF7A11791031708E
:1040A00090F22312263911B390F2231226391232DC
:1040B0004680F51227E87BFF7A1F7920121641E42B
:1040C00090F118F090F118E0FFC3940A5054EF7586
:1040D000F002A424E0FFE5F034BF5156FE740193D2
:1040E000FF90F115123192245CF9E43AFAA3E0FD55
:1040F000315F1225C290F12CEDF090F11512319242
:10410000125FE7ED316212379A784612027790F12A
:104110002D12084E7BFF7A1F79381237C0E004F069
:1041200080A290BFF4E493FE740193FF90F1151206
:1041300026399000701225C290F1151226391235D9
:10414000ACE4120319E4FBFA793078471227827A3B
:104150001F7951021641245CF9E43AFAA3E0FF7595
:10416000F002A4F58285F08322F0A374FFF0A3226D
:104170001216417BFF7A1079660216417BFF7A1096
:1041800079581216417BFF2290F126EFF0A3EDF053
:10419000A3747F3169742AF0A374AAF0E4A3F0A396
:1041A000F0C2AF90F223122639F1CFC3947BE5F031
:1041B0009400503A510A90F12A51129E500851220F
:1041C0007002510380F0510A12A4A5FFC390F12997
:1041D000E09FFF90F128E09EFE51179E502290F143
:1041E00027E0FF90F32051437002510380DA510A17
:1041F00090F12851129E500851227002510380F014
:10420000D2AF2290F12CE004F022E490F12CF0A344
:10421000F022E0FEA3E0FFC390F12DE09F90F12C8F
:10422000E02290F127E0FF90F126E0FD3395E0FCDD
:1042300090F31775F003ED1208AFEC75F003A425A9
:1042400083F583A3E0FAA3E0F5828A83120925901F
:10425000F12DE004F0228F82F583E493221227E807
:10426000E4A3F0A3F0A3F0A3F090F11512263971A6
:10427000392407FDE435F0FC8D82F583E493FF5487
:104280000190F118F0EF5402A2E713A3F08D828C95
:1042900083E493FF5404FEA2E713A2E71390F11AFC
:1042A000F0EF5408FF7803A2E713D8FB90F11BF05E
:1042B00090F1151226391236617BFF7A1E792E1283
:1042C000276712263971392404FFE435F05156125C
:1042D00035347A1E794B1227671226397139240535
:1042E000FFE435F051561235347A1E79641227678F
:1042F00012263971392406FFE435F051561235344F
:104300007A1E797D1216417BFF7A1E799690F118FC
:1043100071487BFF7A1E79AE90F11971487BFF7A64
:104320001E79C690F11A71487BFF7A1E79DE90F1F2
:104330001BE090F12CF00216419000BB0206AE7B10
:10434000FF7A1579C290F125E090F12CF002164128
:104350001227E81230374002A13890F115122639A1
:10436000F1CFFF90F11812366B9000381225CB90E8
:10437000F11AEEF0A3EFF090003A1206AEFD90F1C4
:104380001C123F0C90003C1206AEFD90F11E123F35
:104390000CF1E990F124F0F1EF90F125F01237CD16
:1043A000FD90F122123F0C1237D3FD90F120123F05
:1043B0000C90F161E0D3648094814004E4F08001CA
:1043C0000090F118E0FCA3E0FDF1FE90F11512263B
:1043D0003990005B1205AF30E01B30000B7BFF7A99
:1043E00015799190F1247148C292C29690F124E01F
:1043F000FD7F02A11BD390F119E0942990F118E000
:1044000094005013F1DC300008FB7A1579AB1216DA
:1044100041D17F7F03A11BC390F119E0949A90F1E1
:1044200018E09409400A300002713F12A473A11BE6
:10443000C390F121E0943490F120E09433400E9049
:10444000F11BE0943490F11AE09433500A300002EA
:10445000713F12A473A11BD390F11BE0946690F1FD
:104460001AE09436500E90F123E0946690F122E029
:1044700094364017300007F1D590F1247148C2926C
:10448000D29690F124E0FD7F01A11B90F11EE0FE89
:10449000A3E0FFD390F11DE09F90F11CE09E403D12
:1044A00090F12412A49C6013F1DC300008FB7A1513
:1044B00079AB121641D17F7F03806090F160745414
:1044C000F090F124E090F15FF0300004F1D57148F4
:1044D000C292D29690F15FE0FD7F01803E90F1257F
:1044E000F1F56013F1DC300008FB7A1579AB121698
:1044F00041D17F7F03802490F1607442F090F125D8
:10450000E090F15FF03000087BFF7A1579C27148C6
:10451000D292C29690F15FE0FDE4FF318890F160A5
:10452000E0FDA3123CD412A467F090F15F12A458EE
:1045300090F161E004F0C2B7221227E8E4A3F0A3EF
:10454000F090F323E0D394024002C17E90F1151263
:1045500026399000B91206AEAEF0C3EE94B85004FE
:1045600078137601C3EE94B45004E47813F678130C
:10457000E6146046046002C11AE912A3CA12263981
:104580009000B91225CB12A3D87F0412239050F9C2
:1045900090F115122639123C0E713912A43F71396F
:1045A00064207004E5F064B06002C1541237D97F12
:1045B000041223905002C15480F5125FD412A3CA92
:1045C0001226399000B91225CB12A3D87F041223EA
:1045D0009050F990F115122639123C0E713912A43F
:1045E0003F7139C394E0E5F094B7400E90F1151295
:1045F00026399000B974B0125E8690F115122639F2
:10460000713964207004E5F064B470487D0112379C
:10461000DB7F04122390403C80F7125FDD7F0412A1
:10462000239050F97D02125FDF7F0412239050F92E
:1046300090F11512263912A1F57BFF7A1D79E91246
:1046400016417BFF7A1D79EF1216417BFF7A1E79A6
:104650000E12164190F1151226391236617BFF7A3F
:104660001E79131227671226399000B91236647B1F
:10467000FF7A1D79CC12164190F323E004F022D288
:1046800092D296E4FD221227E81230374002E1CEA2
:1046900090F11512263990003A1206AEFF90F118EB
:1046A00012366B90003C1206AEFF90F11A12366B78
:1046B000F1CFFF90F11C12366BF1E990F11EF0F191
:1046C000EF90F11FF090F15EE0D36480948140029E
:1046D000E4F090F11512263990005B1205AF30E03E
:1046E0001B30000B7BFF7A15799190F11E7148C247
:1046F00092C29690F11EE0FD7F02E1B1D390F11DD0
:10470000E0942990F11CE09400501412A43230007F
:1047100008FB7A1579AB121641D17F7F03E1B19086
:10472000F11AE0FEA3E0FFD390F119E09F90F11899
:10473000E09E403E90F11E12A49C601412A4323000
:104740000008FB7A1579AB121641D17F7F03806197
:1047500090F15D7454F090F11EE090F15CF0300047
:1047600004F1D57148C292D29690F15CE0FD7F01D0
:10477000803F90F11FF1F5601412A432300008FB65
:104780007A1579AB121641D17F7F03802490F15DB9
:104790007442F090F11FE090F15CF03000087BFF74
:1047A0007A1579C27148D292C29690F15CE0FDE42C
:1047B000FF318890F15DE0FDA3123CD412A467F0B4
:1047C00090F15C12A45890F15EE004F0C2B7229020
:1047D00000360206AE7BFF7A1579B12290F1607443
:1047E0002DF090F15F74FFF0229000A40205AF90CD
:1047F00000AD0205AFE0FF7D42123CE2EF22C3EDC7
:10480000949AEC94094005C2C8C2C922C3EF9466C9
:10481000EE94364005D2C8C2C922D3EF9434EE9448
:10482000335005C2C8D2C922D2C8D2C92290F007DB
:104830001227EBA31226399000AE1205AF54036085
:104840002A90F00D1226391179FED3E5F0940AEE84
:104850009400400C122636123FEF1226391227E23E
:1048600090F00712263974010205DC90F007122639
:104870003911CB1226390227E2E475F001020679DC
:1048800090F0071227EBA31226399000AE1205AF65
:1048900030E42A90F00D1226391179FED3E5F09418
:1048A00096EE9400400C122636123FEF1226391273
:1048B00027E290F00712263974020205DC90F00717
:1048C00012263911CB1226390227E2E41205DC90B8
:1048D000F00D2290F0071227EBA31226399000AEBC
:1048E0001205AF5444602A90F00D1226391179FE5A
:1048F000D3E5F09432EE9400400C122636123FEFCE
:104900001226391227E290F00712263974030205A5
:10491000DC90F00712263911CB1226390227E2C2A9
:10492000B022C2B122C2B422C2B522C2B622C2CBC8
:1049300022C29522C29422C29322C2932222D287FB
:1049400022D2B022D2B122D2B422D2B522D2852232
:10495000D28422D2B622D2CB22D29522D29422D293
:104960009322C28722C2B022C2B122C2B422C2B5EF
:1049700022C28522C28422C2B622C2CB22C2952282
:10498000C29422C29322438F01EF7805C333CE3302
:10499000CED8F98EB3F5B2123CD174BE2FF5827425
:1049A000F1123F138EB7F5B675B110E5B020E2FBFA
:1049B00031BBEF2492FFEE3420FE22AFB4AEB553EC
:1049C0008FFE2231E390F1D2E0FEA3E0FF8EB78F9D
:1049D000B675B110E5B020E2FB31BBEEC313FEEFBC
:1049E00013FF22438F017C007D281206108EB38FA7
:1049F000B22290F1181227EB53E87FD2B7A3740AC2
:104A0000F090F11BE0FFC3648094805002A1BE903F
:104A1000F22AEFF090F1307407F0E4FBFD7F011211
:104A2000247F7F177E00122470D2B70000000000A0
:104A30000000000000000000000000000000000076
:104A40000000000000000000000000000000000066
:104A50000000000000000000000000000000000056
:104A60000000000000000000000000000000000046
:104A70000000000000000000000000D283000000E1
:104A80000000000000000090F22AE0B40D00400297
:104A9000A196904A99F8282873024AC0024AFC025B
:104AA0004B38024B74024BB0024BEC024C28024CC8
:104AB00064024CA0024CDC024D18024D5A024D5AC1
:104AC000C2830000000000000000000000000000A1
:104AD00000000000000000000000000000000000D6
:104AE000000000D28700000000B1F0E5A620E4FB42
:104AF00075A3D0E5CB20E1FBC287A196C28300005D
:104B000000000000000000000000000000000000A5
:104B1000000000000000000000000000000000D2C3
:104B2000B000000000B1F0E5A620E4FB75A3D0E5DD
:104B3000CB20E1FBC2B0A196C283000000000000C0
:104B40000000000000000000000000000000000065
:104B50000000000000000000000000D2B1000000D2
:104B600000B1F0E5A620E4FB75A3D0E5CB20E1FB86
:104B7000C2B1A196C2830000000000000000000046
:104B80000000000000000000000000000000000025
:104B900000000000000000D2B400000000B1F0E509
:104BA000A620E4FB75A3D0E5CB20E1FBC2B4A1961F
:104BB000C2830000000000000000000000000000B0
:104BC00000000000000000000000000000000000E5
:104BD000000000D2B500000000B1F0E5A620E4FB23
:104BE00075A3D0E5CB20E1FBC2B5A196C28300003E
:104BF00000000000000000000000000000000000B5
:104C0000000000000000000000000000000000D2D2
:104C1000B600000000B1F0E5A620E4FB75A3D0E5E6
:104C2000CB20E1FBC2B6A196C283000000000000C9
:104C30000000000000000000000000000000000074
:104C40000000000000000000000000D2CB000000C7
:104C500000B1F0E5A620E4FB75A3D0E5CB20E1FB95
:104C6000C2CBA196C283000000000000000000003B
:104C70000000000000000000000000000000000034
:104C800000000000000000D29500000000B1F0E537
:104C9000A620E4FB75A3D0E5CB20E1FBC295A1964D
:104CA000C2830000000000000000000000000000BF
:104CB00000000000000000000000000000000000F4
:104CC000000000D29400000000B1F0E5A620E4FB53
:104CD00075A3D0E5CB20E1FBC294A196C28300006E
:104CE00000000000000000000000000000000000C4
:104CF000000000000000000000000000000000D2E2
:104D00009300000000B1F0E5A620E4FB75A3D0E518
:104D1000CB20E1FBC293807EC28300000000000034
:104D20000000000000000000000000000000000083
:104D30000000000000000000000000D2930000000E
:104D400000B1F0E5A620E4FB75A3D0E5CB20E1FBA4
:104D5000C29390F22A7409F0803CC28300000000E4
:104D60000000000000000000000000000000000043
:104D70000000000000000000000000000000000033
:104D800000B1F0E5A620E4FB75A3D0E5CB20E1FB64
:104D900090F22A740BF01225D2BF81FA1228BBAC14
:104DA00006AD07123CC1123E15EC8DF01207337FA1
:104DB000811225DBC2B790F11BE014F04101E490B1
:104DC000F22AF0123CC1123E1512064EFFAEF0312F
:104DD00086AC06AD07123CD190F1181226398F82AD
:104DE0008E83123FBC90F22AB1F740D743E880226D
:104DF000439C0275A39122E004F0E0C36480948A8E
:104E00002290F1181227EB2490F9E43AFAA3122722
:104E1000EB90F11812319224A4F1061227EB90F1D5
:104E20001812263B90F1211227EBE4FF90F121129A
:104E3000263912064EFDACF090F11BE0FBA3E475A1
:104E4000F002120638A9F0FAEC8DF012073390F157
:104E50001EE0FBA3E475F001120638A9F0FAEF1288
:104E600005DC90F122E475F0021206220FEFB40A7D
:104E7000BB90F1181231922490F9E43AFAC003C0C1
:104E800002C00190F118A3E0FAA3E024A4F9E43AE7
:104E9000FA90F1271227EBA3740AF0D001D002D0C8
:104EA00003123E1C90F1181226399000901206AEA3
:104EB000FF900032123C189000A21206AEFF900044
:104EC00034123C189000381225CBD1FA9E90003A4B
:104ED0008FF01207529000341225CB900038D1FD8C
:104EE0009E90003C8FF01207529000341225CBD1D7
:104EF000FA9E9000368FF00207529000321206AEF2
:104F0000C39FFFE5F022F9E43AFA90F11E22EFB4D4
:104F10000C004003025057904F1EF8282873024F90
:104F200042024F5D024F78024F93024FAE024FC9CB
:104F3000024FE3024FFA0250100250260250330291
:104F40005047209703025057D287125068000EEE48
:104F5000B42AFAD2B753917FC287025057209703E1
:104F6000025057D2B0125068000EEEB42AFAD2B7EF
:104F700053917FC2B0025057209703025057D2B1CD
:104F8000125068000EEEB42AFAD2B753917FC2B124
:104F9000025057209703025057D2B4125068000EA7
:104FA000EEB42AFAD2B753917FC2B4025057209779
:104FB00003025057D2B5125068000EEEB42AFAD24E
:104FC000B753917FC2B5025057209703025057D272
:104FD000B6125068000EEEB42AFAD2B753917FC2CF
:104FE000B68074309771D2CB125068000EEEB42A9E
:104FF000FAD2B753917FC2CB805D30975AD29511C8
:1050000068000EEEB42AFAD2B753917FC29580475A
:10501000309744D2941168000EEEB42AFAD2B753F6
:10502000917FC294803130972E1166000EEEB42A23
:10503000FA800B3097211166000EEEB42AFAD2B72F
:1050400053917FC293801030970D1168000EEEB41B
:105050002AFAD2B753917FD283E4FE000EEEB40B4E
:10506000FAC28322C283D293C2B7439180C297E42B
:10507000FE22C2B7EFB40C0040022168905083F8C2
:105080002828730250A70250B80250C90250DA0211
:1050900050EB0250FC02510D02511E02512F0251E1
:1050A0004002514C02515DD287116A000EEEB42AC3
:1050B000FA53917FC2872168D2B0116A000EEEB414
:1050C0002AFA53917FC2B02168D2B1116A000EEE64
:1050D000B42AFA53917FC2B12168D2B4116A000E8A
:1050E000EEB42AFA53917FC2B4807DD2B5116A0022
:1050F0000EEEB42AFA53917FC2B5806CD2B6116A13
:10510000000EEEB42AFA53917FC2B6805BD2CB1167
:105110006A000EEEB42AFA53917FC2CB804AD29530
:10512000116A000EEEB42AFA53917FC2958039D2EB
:1051300094116A000EEEB42AFA53917FC29480282B
:10514000D293116A000EEEB42AFA800AD293116A41
:10515000000EEEB42AFA53917FC293800B116A00BD
:105160000EEEB42AFA53917FD283E4FE000EEEB421
:105170000BFAC28322D2B7EFB40C004002610B904D
:105180005186F82828730251AA0251C90251E80237
:1051900052070252260252450252640252830252C0
:1051A000A20252BF0252D80252F1209702610BD2E2
:1051B00083E4FE000EEEB411FAC283D287116800B8
:1051C0000EEEB422FAC2876108209702610BD283E7
:1051D000E4FE000EEEB411FAC283D2B01168000EE4
:1051E000EEB422FAC2B06108209702610BD283E4C8
:1051F000FE000EEEB411FAC283D2B11168000EEEB9
:10520000B422FAC2B16108209702610BD283E4FE96
:10521000000EEEB411FAC283D2B41168000EEEB4DF
:1052200022FAC2B46108209702610BD283E4FE0027
:105230000EEEB411FAC283D2B51168000EEEB4229C
:10524000FAC2B56108209702610BD283E4FE000E1A
:10525000EEB411FAC283D2B61168000EEEB422FA8F
:10526000C2B66108209702610BD283E4FE000EEE05
:10527000B411FAC283D2CB1168000EEEB422FAC286
:10528000CB6108209702610BD283E4FE000EEEB4DE
:1052900011FAC283D2951168000EEEB422FAC295BB
:1052A0008066309766D283E4FE000EEEB411FAC237
:1052B00083D2941168000EEEB422FAC29480493071
:1052C0009749D283E4FE000EEEB411FA1164000E89
:1052D000EEB422FAC2938030309730D283E4FE00DD
:1052E0000EEEB411FA1164000EEEB422FAC29380ED
:1052F00017309717D283E4FE000EEEB411FAC28382
:105300001168000EEEB422FA53917F2290F000EF64
:10531000F00000E4FF000FEFB411FA0000E4FF001A
:105320000FEFB422FA2290F00A1227EBC2987BFF0B
:105330007A0979951216417BFF7A0979C0121641D4
:105340007BFF7A0979D41216417BFF7A0979E5123D
:1053500016417BFF7A0979FA1216417BFF7A0A79A6
:105360000C1216417BFF7A0A79261216417BFF7ACE
:105370000A79471216417BFF7A0A79681216417B37
:10538000FF7A0A79891216417BFF7A0A79B31216DD
:10539000417BFF7A0A79CC1216417BFF7A0A79E5C4
:1053A0001216417BFF7A0B79171216417BFF7A0B9D
:1053B00079421216417BFF7A0B79631216413098BD
:1053C000FD209802612EC298E599B4640FE4FF12A3
:1053D00028EA7F011228EA7F021228EAE599B465DB
:1053E000177D007C02125FE17F0412239050F97B4D
:1053F000FF7A0B7984121641E599B46B1253B3FE10
:10540000E41223FED2997BFF7A0B79A6121641E5AE
:1054100099B46C1A53B3FEE4F5BD75985075BE0C83
:1054200043BD01D2997BFF7A0B79B4121641E599FD
:10543000646270367BFF7A0B79C3125E42EFF01222
:105440002368BF0AEF90F00FE07002612E43918055
:10545000D297D29212A4AD317512A411003098FCEB
:10546000C298E599B41BE612A3E6E5996474703717
:105470007BFF7A0C792B125E42EFF0122368BF0A91
:10548000EF90F00FE07002612E12A4B5D29690F06A
:105490000DE0FF124F0E12A411003098FCC298E5E7
:1054A00099B41BE512A3E6E599646970327BFF7A33
:1054B0000C795D125E42EFF0122368BF0AEF90F0A4
:1054C0000FE07002612E12A4B512A4AD117212A4E5
:1054D00011003098FCC298E599B41BEA12A3E6E5E6
:1054E00099647270387BFF7A0C79961216411226F5
:1054F0003612A1F512263612A2F7122636124539B7
:1055000012263612A1F512263612425D12A411009F
:105510003098FCC298E599B41BE612A3E6E59964BD
:105520007370411226361240B37BFF7A0C79B912A0
:10553000164112261A9000AE1205AFC330E301D314
:105540007F0040027F01EF60091236721226361288
:10555000264212A411003098FCC298E599641B7091
:10556000C812A3E6E599646D6002C18F1226361257
:1055700040B37BFF7A0C79CB1237C07401F0A3746F
:10558000F0F0A3740EF07BFF7A0C79F5125E59EF00
:10559000F0122368BF0ADB90F00FE07002612E7BEF
:1055A000FF7A0C79F8125E42EFF0122368BF0AEF1F
:1055B00090F00FE07002612E439180D2977BFF7ACA
:1055C0000D792712164112261A9000AE1205AFC3AC
:1055D00030E301D37F0040027F01EF7002C17B12F4
:1055E000264290F00EE02497605824F5603824128B
:1055F000706F12318F245B12308E54FE1205DC1254
:1056000026369000387430125E8690003274301264
:105610005E86900034743075F000125E7E90F00D5E
:10562000E09000AD803612318F245B12308E54FE34
:105630001205DC122636125E6090F00DE09000A498
:10564000801A12318F245B12308E44011205DC1255
:105650002636125E6090F00DE09000A41205EE80F8
:10566000097BFF7A0D794912164112A028122636BD
:10567000D20012435012262812264212A4110030E2
:1056800098FCC298E599641B6002A1B812A3E6E5F4
:1056900099647570451226361240B37BFF7A0D79F6
:1056A0005012318C245B12308E54FE1205DC12260F
:1056B000159000AE1205AFC330E301D37F00400266
:1056C0007F01EF6015122642122636D2001246865E
:1056D000C298E599B41BD712A3E6E5996476703FAA
:1056E0001226361240B37BFF7A0D797912318C2461
:1056F0005B12308E54FE1205DC1226159000AE129D
:1057000005AFC330E301D37F0040027F01EF600F9C
:1057100012264212263612A47FB41BDD12A3E6E540
:105720009964796002E1F01226361240B37BFF7A69
:105730000D79A2121641439180D297122636123764
:105740003612263612A03812263612A05690F03C99
:10575000EEF0A3EFF090F03CE0FCA3E0FD1237A0E8
:1057600078431227827A0D79CF12164190F03CE0EF
:105770007002A3E060087F021228EABF0108122627
:105780003690005B80241226361237C7FF90F03D1A
:10579000E0241FFD90F03CE03400FCC3EF9DE5F0F9
:1057A0009C90005B400474018001E41205EE122617
:1057B0003690005B1235317A0D79E71216417BFF86
:1057C0007A0E79061216411226289000AE1205AF05
:1057D000C330E301D37F0040027F01EF6012122645
:1057E0004212263612A47F641B6002E13612A3E641
:1057F000E599646160030259B17BFF7A0E790F125B
:105800001641122636123037400221B1E490F00DD5
:10581000F07BFF7A0E792612164190F00DE075F0BC
:1058200004A42410F974F035F0FA90F11874011200
:1058300027ECD124D159EFD10CE599B461DC7BFF81
:105840007A0E7949F180F189501112318FF1E7EF29
:105850001241627440D186D10D80EB122636900041
:105860007074B0D186E490F00DF0122636F1061275
:1058700026361249F2D10DE0C3940240ED122636CD
:10588000123797784312027790F0C012084E90F0CA
:10589000C012375BFB90F038B1EA12027790F0C487
:1058A00012084E7BFF7A0E794BD1C690F0C4B1EA54
:1058B000B1F61226361235ACE412031990F0C41278
:1058C000375BD11490F0DEEEF0A3EFF090F0DCD176
:1058D0009A90F00DF0F1895075EF25E025E0241045
:1058E000F582E434F0B1E8D137F1C7E434F0F58360
:1058F00012084E122636A3E012415F12379AD132B7
:1059000090F00DE0FBF1BBF58312084EEBF1BB12FA
:105910003759FBF1C7E434F0B1E8120277D1ADF5A5
:1059200083F19C90F00DE090F12CF0D1B1B1E8B191
:10593000F6D1ADB1E8E4FBFA79807846D11590F064
:105940000DE0F1A6F583EEF0A3EFD10C8087D1A195
:10595000F1926004EFB46EF6EFB479087B017AF04F
:1059600079C8D1CD1226361240B3E490F00DF01272
:10597000318F1241561206AEFDEFF1A6123F146DA3
:105980007003EE65F0600C7BFF7A0E798590F00D68
:10599000124348D10DE0C3940A40D4122636F15E7A
:1059A00090F0DCE065F07003A3E06F6002F177F146
:1059B0006EE5996467600241BA1226361240B3124E
:1059C000263690007074B0D186F10612263690000B
:1059D000301236647BFF7A0E79D4121641122636C5
:1059E00012379778431227827A0E79E5F1807BFF90
:1059F0007A0E79F61237C07401F0A374F0F0A37434
:105A000044F0D124D159D18C790F90F044B1EA906F
:105A1000F12CB1F9122368BF0AD490F00FE07006A0
:105A200090F00DE014F0D10DE0C3940140C01226B7
:105A300036123797784312027790F03C12084E9056
:105A4000F03C12375BFB90F044B1EA12027790F021
:105A500040D1BD90F040B1EAB1F61226361235AC15
:105A6000E412031990F04012375BD11490F05EEE0F
:105A7000F0A3EFF090F05CD19A90F00DF012318F1E
:105A80001241561206AEFDEF25E02448F582E434BB
:105A9000F0F583E5F0F0A3EDD10CE0B40ADFD1A17D
:105AA000F1926004EFB46EF6EFB479087B017AF0FE
:105AB0007948D1CD1226361240B3E599646360036C
:105AC00002532E7BFF7A0F792B12164112263612C3
:105AD0003037400302532EE490F112F0F1B0501C25
:105AE00012318F245CF9E43AFAEF123CD6123E15DB
:105AF000744075F000120733D12B80E012263690E7
:105B0000007074B0D186E490F10EF0A3F012263646
:105B1000F1061226361249F290F10FE004F07006F9
:105B200090F10EE004F0C390F10FE0940290F10EBA
:105B3000E0940040D8122636124E01122636123C4E
:105B40001F122636123672122636122642E490F1C1
:105B500012F07BFF7A0E79F61237C07401F0A3744D
:105B6000F0F0A37494F0D124D159D18C790F90F036
:105B700094B1EA90F12CB1F9122368BF0AD490F0E5
:105B80000FE0700690F112E014F0D12BE0C36480B6
:105B9000948140BE122636123797784312027790CE
:105BA000F0F012084E90F0F012375BFB90F094B1D9
:105BB000EA12027790F0F4D1BD90F0F4B1EAB1F6B8
:105BC0001226361235ACE412031990F0F412375B4A
:105BD000D11490F110EEF0A3EFF090F10CD19A9067
:105BE000F113F07BFF7A0F794290F1131243489042
:105BF000F113D102C333CE33CED8F9243CF974F07B
:105C00003EFA90F11874011227ECD124D159D18CAD
:105C1000790F90F113D102C333CE33CED8F9243C9F
:105C2000F58274F0B1E790F12CB1F9122368EF64BA
:105C30000A70B090F00FE0700690F113E014F0904D
:105C4000F113124DF7409CE490F112F090F112E044
:105C5000F9C36480948A4002A170E9D103C333CEB2
:105C600033CED8F9243CF58274F0B1E7D137C004C3
:105C7000C005C006C00790F112E0FB3395E0FAEBD7
:105C8000AE027802C333CE33CED8F92468F58274DD
:105C9000F03EF583D007D006D005D00412084EEBB5
:105CA00025E0FFEA33FE1226368F828E8312379A62
:105CB000D132C004C005C006C007B1FFC333CE3324
:105CC000CED8F9FBAA062498F58274F03AF583D071
:105CD00007D006D005D00412084E74982BF58274B4
:105CE000F03A123759FBC000C001C002C003B1FF37
:105CF000C333CE33CED8F92468F58274F0B1E7D03F
:105D000003D002D001D000120277C004C005C00643
:105D1000C007B1FFC333CE33CED8F9D1933EF5835C
:105D2000D007D006D005D004F19C90F112E0FF908E
:105D3000F12CF0D104C333CE33CED8F9D193B1E7EF
:105D4000B1F6B1FFC333CE33CED8F9D193B1E7E486
:105D5000FBFA79807846D115AD07AC0690F11212A6
:105D60003CD4F1663EF583ECF0A3EDF0D12B814CF1
:105D7000D1A190F114EFF064796004E0B46EF19079
:105D8000F114E0B479087B017AF079F8D1CD1226CC
:105D9000361240B3E490F112F0F1B0503112318F6D
:105DA000245CF9E43AFAEF123CD6123E1512064E84
:105DB000FDF166123F136D7003EE65F0600C7BFF22
:105DC0007A0E798590F112124348D12B80CB12269E
:105DD00036F15E90F10CE065F07003A3E06F6002B5
:105DE000F177F16E02532E3EF583E0FCA3E0FDA3B4
:105DF000E0FEA3E0FF2290F12D12084E0216419022
:105E0000F112E0FF3395E0FEEF780222F090F00D02
:105E1000E004F022FB12016EE4FBFAF9783F120075
:105E20007D0203527BFF7A0E79462290F112E00444
:105E3000F02278451202777B9D7A46790278C0027B
:105E4000007D12164190F1187401F0A374F0F0A3D4
:105E5000740DF07BFF7A0B79F8121AE690F00F229E
:105E6000900038743975F0991207529000327439E5
:105E700075F099120752900034743975F099120731
:105E800052900036740275F000020752EFF07BFF6B
:105E90007A0F2224C4F58274F022EEF0A3EFF0E42E
:105EA000227BFF7A0E796A12164102236890F00D68
:105EB000E025E025E02494F582E434F02212084E37
:105EC0007BFF7A0F791C90F12C740AF0221227E8DC
:105ED0007D007C02F1E17F0412239050F9F1D4AEF1
:105EE00002FF12A3AE7FE07EBF12A3D87F0412236D
:105EF0009050F97BFF7A1E79F690F12C74BFF0A3D5
:105F000074E0F002164190F1181227EBE4A3F0A31D
:105F1000F0FFFE90F1181226391224A790F1181202
:105F200026391237C7FF90F11B12366B1224A79047
:105F3000F1181226399000161225CB90F11BE0FCC7
:105F4000A3E0FDC39FEC9E5006AE04AF0580009019
:105F5000F118122639900016EE8FF00207529000C9
:105F6000701206AEFF2274F82FF58274F0227BFFC8
:105F70007A0E79C00216417BFF7A0E79A302164190
:105F8000121641E490F00DF02290F00DE0FFC39462
:105F90000A2290F00EEFF0E0FF64792212084E7BA7
:105FA000FF7A0E795B2225E024C8F582E434F022E2
:105FB00090F112E0FFC36480948A2225E025E0245A
:105FC00068F582E434F02290F00DE025E025E0242D
:105FD0003CF5822290F115A3E0FAA3E0227D017C3A
:105FE00000E4FFFE02002A245CF9E43AFA75F002AC
:075FF0002290003E0207E4CD
:10A00000C3ED9FFFEC9EFED3EF9464EE64809480DA
:10A010007BFF400A7A1079181216417F01227A10CC
:10A0200079371216417F002290F22674FFF0A37454
:10A030002D124169742DF02275DA0475D93C12375E
:10A04000C785F0DCF5DB75D831E5D820E1FB7F076B
:10A050001238297F01221227E8E4FFFDFC75DA049B
:10A0600075D947F5D8E5D820E1FBAFDBEF30E02824
:10A0700075DA0475D944E4F5D8E5D820E1FBACDC09
:10A08000ADDB75DA0475D94775DB0175D811E5D8F4
:10A0900020E1FBAF05AE0422AE04AF052290F1181B
:10A0A0001227EB90003E12088B00000000E490F1B4
:10A0B0001BF090F118123192243EF9E43AFAC003F1
:10A0C000C002C0011207C4C006C00790F11B123CB9
:10A0D000D490F11812263B123EE051E2F8D007D09E
:10A0E0000651EAD001D002D00351D1E0B40AC390A6
:10A0F000F1181226391237C7C4F8540FC868FFE5A3
:10A10000F0C454F048FEE4C006C007125FF1C3D0AB
:10A11000E09FFFD0E09EFE438F01F5B38FB275B78D
:10A120000075B60A75B115E5B020E2FB90F11CE5AB
:10A13000B3F0A3E5B2F0538FFEE490F11BF090F181
:10A140001B125FB3501EA3E0FCA3E0FDEF123CD650
:10A1500090F1181226398F828E83EC8DF01206E66C
:10A1600051D480DA90F11812263990003E12088BF3
:10A1700000000000E490F11BF090F11812319224DD
:10A180003EF9E43AFAC003C002C0011207C4C00697
:10A19000C00790F11B123CD490F11812263B123EDE
:10A1A000E051E2F8D007D00651EAD001D002D00346
:10A1B00051D1E0B40AC3438F0190F118122639122D
:10A1C0005FF1E48EB38FB2125FF1781012079E8EAA
:10A1D000B58FB475B70075B60A75B112E5B020E257
:10A1E000FBAFB2AEB390F1181226399000381225A9
:10A1F000C2538FFE2290F11A1227EBE4FFFEFDFC02
:10A2000090B40051DB6012E4FFFEFDFC90B7E0511A
:10A21000DB7006781776208004E47817F67817E666
:10A2200018F67816E6F9C3648094C15034E9FF3318
:10A2300095E0FEEF7805C333CE33CED8F92400FF86
:10A24000EE34B0FE7814F608EFF6F5828E8312082D
:10A250002EE4FBFAF9F8C312078D60057816068024
:10A26000C17814E6FE08E6FF7003EE64B06008EF04
:10A27000B4001CEEB4B81890F11A1226399000B947
:10A2800074B0125E869000BB74B775F0E0801890D1
:10A29000F11A1226399000B91225C2EF24E0FFEE20
:10A2A00034FF9000BB8FF012075290F11A1226393A
:10A2B0001236617BFF7A1D79B312164190F11A12A2
:10A2C00026399000B91236647BFF7A1D79CC0216CC
:10A2D0004112081490F11BE004F02212083EC30260
:10A2E000078DAEF0FBAA06E4F922EF2BFFEE3AFE53
:10A2F000E93DFDE83CFC221227E890F115122639D1
:10A300009000AE1205AF30E0091247E99000BD128F
:10A3100005EE90F1151226399000AE1205AF30E12E
:10A32000091247EF9000BE1205EE90F11512263982
:10A330009000AE1205AF30E20C9000561205AF90BF
:10A3400000BF1205EE90F1151226399000AE1205ED
:10A35000AF30E40BE924C012308E44011205DC90CA
:10A36000F1151226399000AE1205AF30E60BE92444
:10A37000C012308E44021205DC90F115122639907D
:10A3800000AF1205AF30E00BE924C012308E440458
:10A390001205DC90F1151226399000AF1205AF308E
:10A3A000E10BE924C012308E44081205DC22E4FDE2
:10A3B0000FEFAA0670010E14F5828A83E0FC74C0C8
:10A3C0002DF8A6040DEDB420E72224B9F9E43AFEF5
:10A3D000AF0171AE90F11522AD07AC06ECF5838F9D
:10A3E000827FC002004B7BFF7A0C791D0216417BF5
:10A3F000FF7A1179281216417BFF7A11792D1216F6
:10A40000417BFF7A1179321216417BFF7A11794133
:10A41000227BFF7A0B79FC02164175F003EF1208DC
:10A42000AFEE75F003A42583F583227F007E007DC7
:10A43000002290F15D742DF090F15C74FFF0222405
:10A4400020FFE435F09000B98FF002075290004AE7
:10A450001206AEFF90F12E22E0FD74262FF58274D5
:10A46000F23EF583EDF02274272FF58274F23EF56B
:10A4700083ED22D292C29690F125E0FDE4FF22D234
:10A4800000124350C298E59922FFE43EFEE43DFDF0
:10A49000E43C227F007E007D987CD922E0FF7D5441
:10A4A000123CE2EF2290F12AE0FEA3E022C2969055
:10A4B000F00DE0FF22439180D297C2922290004695
:05A4C0001206AEFF22B0
:00000001FF
